:100000000C94C1010C94E9010C94E9010C94E901F0
:100010000C94E9010C94E9010C94E9010C94E901B8
:100020000C94E9010C94E9010C94E9010C94E901A8
:100030000C94E9010C94E9010C94E9010C94E90198
:100040000C944E150C94E9010C9424140C94FE139A
:100050000C94E9010C94E9010C94E9010C94E90178
:100060000C94E9010C94E9017F0E980E1D0F1E10EF
:10007000421063106F10111000407A10F35A00A064
:10008000724E18090010A5D4E80000E87648170061
:1000900000E40B54020000CA9A3B000000E1F505A1
:1000A000000080969800000040420F000000A086EB
:1000B00001000000102700000000E803000000001D
:1000C0006400000000000A000000000001000000C1
:1000D00000002C76D888DC674F0823DFC1DFAE59DB
:1000E000E1B1B796E5E3E453C63AE651997696E86E
:1000F000E6C28426EB898C9B62ED407C6FFCEFBCF2
:100100009C9F40F2BAA56FA5F490055A2AF75C931C
:100110006B6CF9676DC11BFCE0E40D47FEF520E652
:10012000B500D0ED902E0300943577050080841E35
:10013000080000204E0A000000C80C333333330F90
:10014000986E12831141EF8D2114893BE65516CF2D
:10015000FEE6DB18D1844B381BF77C1D901DA4BB39
:10016000E424203284725E228100C9F124ECA1E5EE
:100170003D273E3E20434F4E464947206D6F646504
:10018000003E3E204D515454206D6F646500537401
:10019000617469632049503A200054797065203FAA
:1001A00020666F722068656C70004448542D4D5174
:1001B00054542041644E6F76656128722920760080
:1001C000444C593D005057443D005553523D004367
:1001D00049443D005356523D004D534B3D00475757
:1001E000593D00444E533D0049503D20004D414390
:1001F0003D002C004448543D005744473D000A55FB
:10020000736167653A0A4F5054494F4E5320536803
:100210006F7720636F6D6D616E647320262070614F
:1002200072616D65746572732076616C7565730AB1
:10023000534156452020202053617665207061721D
:10024000616D657465727320696E746F20454550E9
:10025000524F4D0A4D454D4F5259202053686F77EC
:100260002066726565206D656D6F72790A5645521C
:1002700053494F4E2053686F77206669726D7761DE
:1002800072652076657273696F6E0A0A4B656570D8
:1002900020627574746F6E20646570726573736527
:1002A0006420647572696E6720737461727475700E
:1002B00020746F2064697361626C65206E65747769
:1002C0006F726B20616E64206561736520636F6E71
:1002D00066696775726174696F6E207468726F7594
:1002E0006768205553422E0A0020494E41353D0093
:1002F00020494E41343D0020494E41333D002049C4
:100300004E41323D0020494E41313D0020494E4191
:10031000303D0020484D44543D002054454D503D53
:10032000002F003D0000000000240027002A0000EC
:10033000000000250028002B0000000000230026FC
:10034000002900000000080002010000030407006B
:10035000000000000000000404040404040404027B
:100360000202020202030303030303010204081052
:10037000204080010204081020010204081020001F
:10038000022911241FBECFEFD8E0DEBFCDBF11E0A0
:10039000A0E0B1E0EAE7F3E602C005900D92AE3DC1
:1003A000B107D9F726E0AEEDB1E001C01D92A3364A
:1003B000B207E1F711E0C1ECD1E004C02197FE01E2
:1003C0000E946B31C03CD107C9F70E944C200C94AD
:1003D000BB310C940000CF93DF931F92CDB7DEB7F3
:1003E000DC01ED91FC910288F389E02D41E050E0C1
:1003F000BE016F5F7F4F0995181619061CF489819D
:1004000090E002C08FEF9FEF0F90DF91CF910895A2
:10041000FC01448555854115510551F0FB012485AA
:1004200035852115310521F081E04217530709F088
:1004300080E00895DC011C96ED91FC911D973097AA
:1004400039F08181811106C0808182958170089583
:1004500080E0089581E0089580E090E00895DC0157
:10046000ED91FC91028CF38DE02D099591E08927A7
:100470000895089580E090E00895CF93DF93EC0114
:10048000888181110E949815DE011196FE01CE012E
:1004900004962D912193E817F907D9F71C82DF9173
:1004A000CF9108950F931F93CF93DF93EC018C01AD
:1004B0000B5F1F4F888181110E9498151992C017F8
:1004C000D107C1F7DF91CF911F910F910895CF937D
:1004D000DF93EC01E881F981008CF18DE02D099525
:1004E000882339F08C859D850196DF91CF910C94FE
:1004F0005202DF91CF910895DF92EF92FF920F9316
:100500001F93CF93DF93C09140028C2F8270C1FF65
:100510000FC020913F0230E041E552E060E070E022
:10052000809150020E94FE17CD7FC093400215C0FB
:10053000C091F801D091F901209719F0CE010E94E5
:10054000251780935002882309F471C09E0141E56C
:1005500052E060E070E00E94FE17E091500280914E
:100560007304882309F45AC085E0E89FF001112440
:10057000EA55FC4FC081D1812197028113810C0F74
:100580001D1FCE010E94B416D82E882321F060E0F2
:10059000CE010E949C16BE0184E00E941E16B80186
:1005A00086E00E941E168AE0E82EF12C40E86FE1FA
:1005B00080E80E94D91540E86FE180EA0E94D915D1
:1005C0004AE06CE180EA0E94D91548E06FE180E8DA
:1005D0000E94D91504E610E08CE10E946F168A7023
:1005E00061F40115110559F0015011096AE070E03C
:1005F00080E090E00E940815EFCF012B49F448E01D
:100600006FE180EA0E94D91581E0E81AF10871F6DD
:10061000DD2021F06D2DCE010E949C1680915002AC
:1006200081110E9498151092500281E001C080E073
:10063000DF91CF911F910F91FF90EF90DF90089580
:10064000EF92FF920F931F93CF93DF93EC01E8811A
:10065000F981008CF18DE02D09958823B9F08C8506
:100660009D857C012FEFE21AF20A8C010A5F1F4F71
:10067000C0E0D0E0F70181917F010E948018C80F8F
:10068000D91FE016F106B1F7CE0102C080E090E07C
:10069000DF91CF911F910F91FF90EF900895EF920E
:1006A000FF920F931F93CF93DF9300D0CDB7DEB7A8
:1006B0007C018B0149835A830E944215F701E85758
:1006C000FF4F6083718382839383D70114968D914A
:1006D0009C911597DC01ED91FC910280F381E02D56
:1006E00049815A81B8010F900F90DF91CF911F91EE
:1006F0000F91FF90EF9009941F93CF93DF93EC013C
:10070000162F0E944215FE01E857FF4F6083718348
:10071000828393838C819D81DC01ED91FC9101901A
:10072000F081E02D612FDF91CF911F9109940F93FC
:100730001F93CF93DF931F92CDB7DEB78C01DC01FF
:10074000ED91FC91008CF18DE02D09958823B1F09D
:10075000D8011C96ED91FC911D978181882371F041
:1007600041E050E060E070E00E944518BE016F5F1C
:100770007F4F0E94B615898190E002C08FEF9FEFF6
:100780000F90DF91CF911F910F9108954F925F923B
:100790007F928F929F92AF92BF92CF92DF92EF9211
:1007A000FF920F931F93CF93DF937C014B01EA01DC
:1007B000DC01ED91FC91008CF18DE02D09958823F1
:1007C00009F475C0D7011C96ED91FC911D978181AC
:1007D000882309F46FC06E018EE1782E8E010C190A
:1007E0001D09080D191DD7011C96ED91FC911D974F
:1007F000A60160E070E081810E9445185C01B801AB
:100800000E94B615F70144845584D20111961C91BB
:10081000812F0E948018A816B90681F5CA18DB0836
:10082000C20101960E943D02F701A485B5858C9115
:10083000282F30E02F70729EF001739EF00D11246E
:10084000EB5DFC4F918D94FF05C0982F907611F4CD
:1008500080688C93D7011C96ED91FC911D97818146
:1008600081111FC0808186FF05C010821D961C92D9
:100870001E921C97CE018C199D091EC0B5E01B9FCE
:10088000F0011124EA55FC4F808191818A0D9B1D56
:1008900091838083828193818A199B0993838283C8
:1008A00004C0C114D10409F099CFCE0105C08FEF67
:1008B0009FEF02C080E090E0DF91CF911F910F91F8
:1008C000FF90EF90DF90CF90BF90AF909F908F9070
:1008D0007F905F904F900895CF92DF92EF92FF92BA
:1008E0000F931F93CF93DF9380917304882309F4B0
:1008F0001AC2D0913E02D11162C089E30E946F16E4
:1009000090917304992309F458C0882309F455C0C1
:1009100060917404709175048B010A5F1F4F01157B
:1009200028E0120710F00F5F174080E00E941E16AB
:1009300060E08AE30E944D1690E0909375048093E6
:10094000740460E08AE30E944D1620917404309193
:100950007504382B309375042093740460E08AE3A7
:100960000E944D16C82F60E08AE30E944D16F82EB3
:1009700060E08AE30E944D16E82E40E46EE180E8D4
:100980000E94D9156091740470917504E7FE12C03D
:10099000611538E0730770F41093770400937604C0
:1009A0008C2F90E09F29049790937904809378048A
:1009B000DFEF03C08CE00E941E16D0933E02109120
:1009C0003E02112309F44AC181E080934002812F45
:1009D0000E948018EC019093F9018093F801892B13
:1009E00009F42FC142E650E060E070E0812F0E94E0
:1009F000451861E572E00E94B615E0905D02F09046
:100A00005E0248E0E416F10409F06AC01093500257
:100A10002E97D093F901C093F80120916B02309189
:100A20006C02E091C602F091C702AF014227532742
:100A30008091BE029091BF0284239523892B09F0F7
:100A400042C040916D0250916E026091C802709157
:100A5000C902DB01A427B5278091C0029091C10291
:100A60008A239B23892B79F580916F0290917002E4
:100A70008E179F0771F48091710290917202861710
:100A8000970739F467E572E08BE692E00E94570918
:100A90001AC080E09BE08830A1F0989FF0011124FB
:100AA000E653FD4F608171812617370741F462815B
:100AB00073814617570719F480932203E3CF8F5FA2
:100AC000EACF8093220381E00E94F40A8091F8012A
:100AD0009091F901892B09F4B4C00E94C009AFC0FC
:100AE00058E0E51656E0F50609F0ABC01092F901A2
:100AF0001092F801AA9708F49CC080916502909129
:100B000066028115A1E09A0729F08115924009F447
:100B100074C08FC020917702309178028091C60214
:100B20009091C7022817390709F083C020917902F4
:100B300030917A028091C8029091C9022817390732
:100B400009F077C067E672E08DE692E00E945709EF
:100B500080E092E0909366028093650286E0E7E68B
:100B6000F2E0A1E7B2E001900D928A95E1F786E00C
:100B7000EBE7F4E0A7E6B2E001900D928A95E1F789
:100B800086E0EBE7F4E0A7E5B2E001900D928A95EC
:100B9000E1F786E0E1E7F2E0A1E5B2E001900D9235
:100BA0008A95E1F780916D0290916E0290937802A0
:100BB0008093770280916F029091700290937A02F5
:100BC000809379028091C6029091C70290936E0241
:100BD00080936D028091C8029091C9029093700237
:100BE00080936F02F0925E02E0925D028AE290E0F2
:100BF0009093F9018093F8011CC020917702309105
:100C000078028091C6029091C7022817390789F4AB
:100C10002091790230917A028091C8029091C902A4
:100C20002817390731F467E672E08DE692E00E94FA
:100C300057098091F8019091F901892B11F00E94D8
:100C40007C028091400280FF09C060917404709121
:100C500075048CE00E941E1610923E020E944215FE
:100C60006B017C018091810490918204A0918304A6
:100C7000B0918404A7019601281B390B4A0B5B0B2A
:100C8000DA01C90180959095A095B0958827B7FDA8
:100C900083959927AA27BB27C82F05E213E0109355
:100CA000F7010093F601CC2311F082E017C0011583
:100CB000110519F1D8015C96ED91FC915D97309783
:100CC000D1F085859685A785B089A7019601281B57
:100CD000390B4A0B5B0B57FD10C083E00E94F40AEE
:100CE0008091F8019091F901892B39F00E94C00997
:100CF0000E947C0202C0F801E4CF025E1F4F33E085
:100D00000D39130761F6CC2371F0D701C601865067
:100D10009F4FAF4FBF4F8093810490938204A09365
:100D20008304B0938404DF91CF911F910F91FF90C2
:100D3000EF90DF90CF9008958F929F92AF92BF92E5
:100D4000CF92DF92EF92FF920F931F93CF938C017C
:100D50005B017A016A014C0187E0880E911C0E94B8
:100D60006C040115110509F452C0F80180818076E8
:100D700009F04DC0F401C1E08191811102C0C15060
:100D800004C0CF5FC530C1F7C4E0F801EC0FF11D1E
:100D9000868181110DC080E092E00E942517F80144
:100DA000EC0FF11D86838823D1F2F8011486138697
:100DB000A7014C195D094A0D5B1DF8016385748517
:100DC0009601EC0FF11D86810E94FE17C81AD90A00
:100DD000F80123853485820F931F948783871C1421
:100DE0001D042CF4C43009F4BACFCF5FD4CF0E94D5
:100DF0004215DC01CB010A96A11DB11DF8018587C2
:100E00009687A787B08BC7018C199D0902C080E027
:100E100090E0CF911F910F91FF90EF90DF90CF90D6
:100E2000BF90AF909F908F900895FC018485958529
:100E30000C949C06CF93DF931F92CDB7DEB76983E6
:100E400041E050E0BE016F5F7F4FFC0184859585D6
:100E50000E949C060F90DF91CF910895CF93DF936E
:100E6000EC010E946C04EC85FD85309739F080819F
:100E700086FF06C081E09181911103C080E001C02E
:100E800081E0DF91CF910895CF93DF93EC018C85C2
:100E90009D85009781F0FC012081222361F001965D
:100EA0000E945202EC85FD85908196FF02C010825F
:100EB00002C0906290831D861C86DF91CF910C94B6
:100EC0006C04EF92FF920F931F93CF93DF938C01EB
:100ED0007B01EA01DC01ED91FC910488F589E02DAC
:100EE0000995F701828190E0982F88272381822B32
:100EF000982789279827248130E0322F222745819F
:100F0000242B3227232732277C2F6D2F4091230358
:100F1000509124034F5F5F4F4115FDE75F0710F0CD
:100F200040E050E1D42FC52FE5E2F3E0A0E0A4308B
:100F300059F0B18DBB2329F0E480F580EC16FD0655
:100F400049F3AF5F7E96F3CF50932403409323037E
:100F50001092A50340E0C0E0D0E0AEE14430C1F023
:100F6000A49FF0011124EB5DFC4F518D511104C081
:100F70004093A503EF010EC0573031F4209729F0BC
:100F8000B28D5A8D5B1708F0FE014F5FEF01E6CF7F
:100F90004093A503209719F480E090E040C042E020
:100FA000498F4091EB014C874091EC014D87409176
:100FB000ED014E874091EE014F8740E052E05B8BA0
:100FC0004A8B5D8B4C8B41E050E0598B488B1B8EDC
:100FD0004A8F43E0488F1E8A40E14F8B40912303A4
:100FE000509124035427452754275D834C837F83E6
:100FF0006E83998388833B832A83898D8F7061F206
:101000000E946C04898D8F708330B9F78C8D9D8D13
:10101000D8011D969C938E931C9781E090E0DF9100
:10102000CF911F910F91FF90EF900895AF92BF92D3
:10103000CF92DF92EF92FF920F931F93CF93DF93A4
:10104000E090F601F090F701D7015C96CD91DC912C
:101050005D97D090F5012097B1F5D6FE67C0EAEF15
:10106000F1E080E090E02081211127C041E1489F1C
:101070009001499F300D1124E901C650DE4FA701B0
:1010800045525340559547956FEE7EEE469FC00101
:10109000479F900D569F900D112480618883F90120
:1010A000E550FE4F80E1DF011D928A95E9F7209718
:1010B000E9F1F701D58FC48F06C00196719684308F
:1010C000910589F633C0D1FE08C00091F801109156
:1010D000F9010115110509F04FC0888187FF0AC089
:1010E0008F7788838D2D82608093F501F701818D44
:1010F0008F7E818F1091F501F12FF071BF2E14FFBB
:1011000073C0CE0106960E9452028981882309F499
:101110006EC0D70114968D919C9115979F838E83F5
:10112000888180648883F701158E148EE12CF12C60
:101130006091F3017091F401F092F201E092F101FB
:101140001E141F0454F48091EF019091F001681770
:10115000790719F0A7010E947E31F092F901E0921F
:10116000F801DF91CF911F910F91FF90EF90DF90E9
:10117000CF90BF90AF9008958881807609F0ADCF71
:101180005E01FFEFAF1ABF0AC12CD5018C9181110E
:1011900017C0C8010E942517F5018083882381F0BC
:1011A0002091F3013091F4012155324040913E02EB
:1011B00060E070E00E94C917F4E0CF128ECF0CC03F
:1011C000C394BFEFAB1ABB0AE5E0CE12DECF80912D
:1011D00040028E7F80934002D70159968C91599797
:1011E000806159968C9379CF17FF03C08ACF1882FC
:1011F0009ACF10FF04C0CE0106960E943D021C70DB
:1012000009F440C08E818823E9F19F8191110FC0BC
:10121000EB84FC84E114F10409F48ACF95E0899F02
:10122000F0011124EA55FC4FF382E28206C00E94CD
:1012300080187C01892B09F47BCF6091F3017091B8
:10124000F4016155724060933F026B01DD24C701D8
:101250008C0D9D1D009719F00E942517B82EB09295
:101260005002BB2009F464CF870120E030E04E81BA
:10127000B6018B2D0E94C917809140028260809335
:10128000400256CF888185FF51CF8E8181110AC0DF
:101290001882D7015D961C921E925C9780E1809324
:1012A000F50144CFF701818D8061818F3FCFEF92AF
:1012B000FF920F931F93CF93DF939C01FB0110923A
:1012C000220390E08BE0983031F1899F7001112466
:1012D000E701C653DD4F6881798161157105C9F059
:1012E0004A815B8141155105A1F0D9010D911C91F5
:1012F00011970617170769F412966D917C91139751
:101300006417750731F490932203D701A253BD4FA0
:101310002AC09F5FD8CF90E08BE0983091F0899FF2
:10132000E0011124C653DD4F48815981452B39F422
:101330004A815B81452B19F4909322030AC09F5F79
:10134000ECCF10924B0210924A0210922203CAEC88
:10135000D2E0D9014D915D916D917C91DE014D936B
:101360005D936D937D9386E001900D928A95E1F7F0
:101370001A86DF91CF911F910F91FF90EF90089502
:10138000CF93DF9300D000D000D0CDB7DEB78091EF
:101390006F02909170028F3F2FEF920759F42091C6
:1013A0007102309172022F3F3F4F21F486E0EAE054
:1013B000F1E0F3C02091C6023091C70228273927F7
:1013C0004091BE025091BF0224233523232B91F478
:1013D00060917102709172022091C8023091C9022D
:1013E000262737274091C0025091C102242335237C
:1013F000232B89F08091C2029091C30290934D02F9
:1014000080934C028091C4029091C50290934F0248
:1014100080934E0208C090934D0280934C027093CB
:101420004F0260934E0220914C0230914D02409148
:101430004E0250914F0280E09BE08830B9F1989FB6
:10144000D0011124A653BD4F6D917C9111972617A1
:10145000370751F512966D917C91139746175707F0
:1014600019F5FD01349614966C911497611118C00A
:1014700015966C911597611113C016966C9116977D
:1014800061110EC017966C911797611109C01896DB
:101490006C911897611104C019966C91662321F024
:1014A0008093220386E079C08F5FC7CF80932203A9
:1014B00046E050E06FEF70E081E592E00E949931E4
:1014C00086E0E1E7F2E0DF01282F1D922A95E9F797
:1014D000EBE7F4E0A7E5B2E0982F01900D929A9522
:1014E000E1F7EBE7F4E0A7E6B2E0982F01900D9268
:1014F0009A95E1F720914C0230914D023093780299
:101500002093770220914E0230914F0230937A025D
:10151000209379022091C6023091C70230936E0267
:1015200020936D022091C8023091C902309370025D
:1015300020936F0220E031E0309366022093650231
:101540003093600220935F0228E030E03093620223
:10155000209361028093630294E09093640228E0F8
:1015600036E030935E0220935D0227E832E030934C
:10157000F4012093F3012AE230E03093F901209343
:10158000F801BE016F5F7F4FDB011D928A95E9F77D
:101590008CE492E00E9457091EC0A1E5B2E00190E0
:1015A0000D928A95E1F786E0EBE7F4E0A7E5B2E07B
:1015B00001900D928A95E1F788E090E090935E02A9
:1015C00080935D028091F8019091F9010E969093BD
:1015D000F9018093F80126960FB6F894DEBF0FBE8E
:1015E000CDBFDF91CF910895FF920F931F93CF93BB
:1015F000DF93C091F601D091F70127E832E03093F4
:10160000F4012093F3013093F0012093EF01833034
:1016100059F4898D8F70833009F0FBC588899989C9
:10162000892B09F0F6C57EC0823009F07FC0809119
:10163000EE018F5F8093EE01811113C08091ED0167
:101640008F5F8093ED0181110CC08091EC018F5F61
:101650008093EC01811105C08091EB018F5F809335
:10166000EB011092F9011092F8011092F201109220
:10167000F101898D982F9D7F953041F48A8D8F5F80
:101680008A8F883709F0C5C5198EC3C5882309F428
:10169000C0C528893989232B09F440C09A8D2FEFC2
:1016A000290F2A8F9111B5C59B8D983031F02FEFFE
:1016B000280F223048F4953039F4198E80E8809351
:1016C000F5010E94160851C4953038F423E0092E24
:1016D00001C0220F0A94EAF701C020E32A8F9F5F1E
:1016E0009B8F8F708330A1F048F4813009F42BC2B6
:1016F000823009F08EC51092800228C2863009F42B
:1017000043C4883009F440C4843009F082C53CC425
:1017100084E08093F5010E9416085CC48F708330CA
:1017200009F077C588E08093F50114C480915F02C9
:10173000853409F06EC58091610290E0982F88276A
:1017400020916202820F911D2091F8013091F901E0
:101750002817390708F45DC59093F9018093F801C3
:10176000809165028F7309F054C5F0906602F11004
:1017700050C5C091C602D091C702209731F4809124
:10178000C8029091C902892BA1F080916F029091BB
:1017900070028C179D0709F03CC5209171023091B1
:1017A00072028091C8029091C9022817390709F086
:1017B00030C50E941E19019609F02BC58091680260
:1017C0008630B1F1813009F024C5809173028830F0
:1017D00009F01FC5109273028091750290917602F4
:1017E000873F4FEF940710F0099601C00896909339
:1017F00076028093750280916B0290916C029093B7
:10180000700280936F0280916D0290916E029093AE
:10181000720280937102D0936C02C0936B0280912C
:10182000C8029091C90290936E0280936D02F5C434
:101830000E949918019609F0ECC42091750230912C
:101840007602809173029091740260916B027091A4
:101850006C02E0916D02F0916E0205E213E0D80196
:1018600059964C9159974423C1F014960D90BC9110
:10187000A02D2A173B0789F4E801AE81BF818A17A2
:101880009B0759F4A881B9816A177B0731F4AA81B3
:10189000BB81EA17FB0709F470C1025E1F4FD3E05A
:1018A0000D391D07E1F6809180028F738230E1F4DB
:1018B000309349022093480280E0843099F0E82F69
:1018C000F0E0EE0FFF1FE356FC4F408151818F5F28
:1018D0002417350791F71092A50380E0C0E0D0E00F
:1018E0009EE17CC08093A5038091800282FD91C41B
:1018F00084E18093800288E290E09093F9018093E4
:10190000F80180E580937F0230917A0280917E0217
:1019100080937A022091790280917D0280937902EE
:1019200020937D029091780280917C0280937802CE
:1019300090937C02809177028093A50340917B0273
:101940004093770280937B023F5F30937E02311198
:101950000DC02F5F20937D02211108C09F5F9093DF
:101960007C02911103C08F5F80937B028091730290
:1019700090917402909349028093480220917502DD
:101980003091760230937402209373029093760222
:101990008093750280916B0290916C02909370021B
:1019A00080936F0280916D0290916E02909372020B
:1019B000809371028091C6029091C70290936C024D
:1019C00080936B028091C8029091C90290936E023D
:1019D00080936D02E0C3473099F08F5F8430F1F05F
:1019E000282F30E0929FF001939FF00D1124EB5DC2
:1019F000FC4F418D4111EFCF8093A503EF0110C043
:101A0000209721F0528D4A8D451738F7929FE001BB
:101A1000939FD00D1124CB5DDC4FDFCF8093A503C6
:101A2000209709F4F6C3D093F701C093F60183E041
:101A30008A8F888F1E8A84E08F8B1B8E809175021F
:101A4000909176029D838C838091730290917402B1
:101A50009F838E8380916B0290916C02998388831F
:101A600080916D0290916E029B838A8381E0898FC1
:101A70008091EB018C878091EC018D878091ED0145
:101A80008E878091EE018F8781E090E0998B888B23
:101A900080917A028B87809179028A87809178027F
:101AA000898780917702888781E090E00E94E5280D
:101AB00080917F02982F907F913508F444C08295E1
:101AC0008F7090E00597880F991F880F991F2091BC
:101AD0004702EF2DF0E0E817F9078CF5EF5AFD4FBC
:101AE00026A9211105C0F092A503109247022BC030
:101AF000213011F4F394EDCF2230E1F437A93430E2
:101B0000C9F4F092A5032093470280AD90E0982F8E
:101B1000882721AD822B909349028093480281301F
:101B2000E2E09E0710F080E092E09B8B8A8B9D8B19
:101B30008C8B09C037A9332311F0F30ECACFF09272
:101B4000A5032093470280E1809380028091800268
:101B500082608093800282E08093870294E0909379
:101B600088028093890210928A028CE290E090931E
:101B7000F9018093F80180E6BCC2E8011093F701F7
:101B80000093F6011092F50130918002F32FF4706A
:101B9000FF2E32FF03C0198E80E24BC220917F02DC
:101BA00022952F70220F220F2093A5038091F80118
:101BB0009091F9014497821B91099093F9018093C8
:101BC000F8014F70423021F4232F2F73223109F195
:101BD000892B19F4832F8370E1F090917702D8015B
:101BE00018968C91189798137AC29091780219964A
:101BF0008C911997981373C2909179021A968C91CF
:101C00001A9798136CC290917A021B968C91981334
:101C100066C234FF63C0F80160897189611571057E
:101C200009F45CC0C8010C960E94AF2830917B0279
:101C300080914302381352C020917C02809144026B
:101C400028134CC090917D0280914502981346C0A4
:101C500080917E0240914602841340C0D8011C96B8
:101C60003C931C971D962C931D971E969C931E9734
:101C70001F968C931F975B968C915B97811126C062
:101C800056969C91569758968C9158975A962C91A7
:101C90005A97821B292F269526952695821B980FE9
:101CA00056969C93569787FD819557962C915797FA
:101CB000322F36953695231B820F57968C93579764
:101CC000969596959695890F58968C9381E080937A
:101CD000F501F801808D828F118A108AD8015996FA
:101CE0002C91E22FEF708E2F90E0FC013197E830BD
:101CF000F10508F08EC2EC5CFF4F0C946B318091C3
:101D0000F50180FF86C283E0F801818F80E4809333
:101D1000F501118A108A8091F8019091F9010097DC
:101D200009F414C122E42093F5010E94E5280EC1B4
:101D30008091F50180FF76C0809180028F7382319F
:101D400009F070C080917F02982F907F913508F440
:101D500049C082958F7090E00597880F991F880F72
:101D6000991F20914702EF2DF0E0E817F907B4F52D
:101D7000EF5AFD4F26A9211105C0F092A50310923C
:101D8000470230C0213011F4F394EDCF223009F531
:101D900037A93430F1F4F092A5032093470280ADC7
:101DA00090E0982F882721AD822B90934902809351
:101DB00048028130F2E09F0710F080E092E0D80105
:101DC00053969C938E93529755969C938E935497CB
:101DD00009C037A9332311F0F30EC5CFF092A50344
:101DE0002093470283E0F801818F809177028087FA
:101DF00080917802818780917902828780917A022E
:101E0000838781E090E00E94E52882E48093F501D9
:101E1000D80151961C921E9250971092F90110927F
:101E2000F80194C080E28093F5010E941608E091C9
:101E3000F601F091F701118E57CD8091800280FF5D
:101E40002EC024FD2CC0F80180899189892B09F0CE
:101E5000E0C18091F8019091F90101960E94E52876
:101E60008091F501982F90619093F5012091F801F0
:101E70003091F901232B19F082618093F5010E94C2
:101E8000160881E090E0D80151969C938E9350976C
:101E900088E059968C9359975B961C9275C085FF84
:101EA0001DC08091850290E0982F8827309186028E
:101EB000832B4091F3015091F401480F591F509327
:101EC000F4014093F3014091F8015091F901FA01B6
:101ED000E81BF90BF093F901E093F8014091F80148
:101EE0005091F9014115510551F024FD08C0909120
:101EF000F50192609093F501CA010E94E528809156
:101F0000810290E0982F882720918202820F911DF4
:101F10009093490280934802D80154962D913C91A8
:101F200055972817390710F0892B21F4309349026F
:101F3000209348028091480290914902F801938BC6
:101F4000828B8091F501837009F463C11092F201D4
:101F50001092F1010E9416088091F50185FF07C0DB
:101F60001092F2011092F101198E84E1B9C084FF40
:101F70000DC01092F2011092F10181E090E0998B76
:101F8000888B84E0898F1B8E81E1AAC02091F101AA
:101F90003091F20121153105E1F080FF02C0198A6C
:101FA000188A88899989009781F48A899B89821780
:101FB000930720F49093F2018093F1018091F10155
:101FC0009091F201998B888B04C09093F2018093D9
:101FD000F1011B8E8091EF019091F0019093F4013B
:101FE0008093F3018091F1019091F201892B59F0D6
:101FF00088899989009739F088969093F9018093A0
:10200000F80188E10BC08091F50181FF02C188E2EF
:1020100090E09093F9018093F80180E18093800231
:1020200067C08091F50180FFF4C0D80159961C92D9
:1020300080E18093F5010E941608EBC08091F801C1
:102040009091F901009711F00E94E528909180028B
:102050008091F50190FF0EC080FF07C087E0F80176
:10206000818F128E118A108A1DC086E0D801599680
:102070008C9318C080FF20C085E0E801898F198A01
:10208000188AC7C08091F8019091F901009711F06A
:102090000E94E5288091800280FF0EC087E0F80151
:1020A000818F128E81E090E00E94E52880E180938C
:1020B000F5010E94160813C08091F8019091F90172
:1020C000892B69F4A6C08091F50180FFA2C087E04A
:1020D000D80159968C9359975A961C929AC080E1D0
:1020E0008093800288E290E09093F9018093F80158
:1020F00080E580937F02888580937B028985809329
:102100007C028A8580937D028B8580937E028C85FC
:10211000809377028D85809378028E8580937902F3
:102120008F8580937A0286E0809368028C819D81FE
:1021300090937402809373028E819F8190937602B4
:10214000809375028091C6029091C70290936C02B1
:1021500080936B028091C8029091C90290936E02A5
:1021600080936D02888199819093700280936F02B1
:102170008A819B819093720280937102898D84FF82
:1021800005C0109282021092810205C082E0809305
:1021900081021092820280E4809367028091F801AC
:1021A0009091F901909361028093620210928602ED
:1021B0001092850210928402109283020E94991854
:1021C00080959095909384028093830285E4809318
:1021D0005F02109260021092660210926502809176
:1021E00041029091420201969093420280934102F3
:1021F000909363028093640210926A0210926902C3
:102200000E941E198095909590936A0280936902AE
:1022100004C01092F9011092F8011092F501DF91BB
:10222000CF911F910F91FF9008950F931F93CF931C
:10223000DF938C01C62F660FDD0B60E575E0CE01E4
:102240000E94B43165EB71E0CE010E94A031B8016B
:10225000CE010E94A031CE01DF91CF911F910F914D
:102260000895CF92DF92EF92FF920F931F93CF9337
:10227000DF93CDB7DEB72C970FB6F894DEBF0FBE55
:10228000CDBF7C018B01FB01E40FF51F10820E9482
:102290008C1F83E293E00E94911FC8010E940920D5
:1022A000CE0101966C01682F87E991E00E9415111B
:1022B000BC01C7010E94AB31892B39F4C8010E94CF
:1022C000612B682F83E00E947F146C2D8CE991E0D4
:1022D0000E941511BC01C7010E94AB31892B39F452
:1022E000C8010E94612B682F84E00E947F146C2D2E
:1022F00081EA91E00E941511BC01C7010E94AB3137
:10230000892B39F4C8010E94612B682F85E00E9457
:102310007F146C2D86EA91E00E941511BC01C70163
:102320000E94AB31892B39F4C8010E94612B682FC0
:1023300086E00E947F146C2D8BEA91E00E941511BB
:10234000BC01C7010E94AB31892B39F4C8010E943E
:10235000612B682F87E00E947F146C2D80EB91E049
:102360000E941511BC01C7010E94AB31892B39F4C1
:10237000C8010E94612B682F88E00E947F142C9670
:102380000FB6F894DEBF0FBECDBFDF91CF911F9186
:102390000F91FF90EF90DF90CF900895CF92DF9252
:1023A000EF92FF920F931F93CF93DF936C017A010B
:1023B0008B01C0E0D0E0CE15DF0589F0D8016D912A
:1023C0008D01D601ED91FC910190F081E02DC601C7
:1023D0000995892B11F47E0102C02196ECCFC7012B
:1023E000DF91CF911F910F91FF90EF90DF90CF90F1
:1023F0000895FC01538D448D252F30E0842F90E00B
:10240000821B930B541710F0CF96089501970895EF
:10241000FC01918D828D981761F0828DDF01A80FEC
:10242000B11D5D968C91928D9F5F9F73928F90E00E
:1024300008958FEF9FEF0895FC01918D828D98177D
:1024400031F0828DE80FF11D858D90E008958FEFBA
:102450009FEF0895FC01918D228D892F90E0805C83
:102460009F4F821B91098F739927089586E894E006
:102470000E942A1221E0892B09F420E0822F08957E
:10248000FC01848DDF01A80FB11DA35ABF4F2C9111
:10249000848D90E001968F739927848FA689B789E0
:1024A0002C93A089B1898C9180648C93938D848DB9
:1024B000981306C00288F389E02D80818F7D808388
:1024C0000895EF92FF920F931F93CF93DF93EC0148
:1024D00081E0888F9B8D8C8D981305C0E889F989E0
:1024E000808185FD24C0F62E0B8D10E00F5F1F4FFD
:1024F0000F731127E02E8C8DE8120CC00FB607FC6D
:10250000FACFE889F989808185FFF5CFCE010E9455
:102510004012F1CF8B8DFE01E80FF11DE35AFF4F02
:10252000F0820B8FEA89FB898081806207C0EE8987
:10253000FF896083E889F98980818064808381E0F4
:1025400090E0DF91CF911F910F91FF90EF90089550
:10255000CF93DF93EC01888D8823C9F0EA89FB894A
:10256000808185FD05C0A889B9898C9186FD0FC041
:102570000FB607FCF5CF808185FFF2CFA889B98916
:102580008C9185FFEDCFCE010E944012E7CFDF9105
:10259000CF91089580E090E0892B29F00E943612B7
:1025A00081110C94000008953FB7F8948091BA020D
:1025B0009091BB02A091BC02B091BD0226B5A89B30
:1025C00005C02F3F19F00196A11DB11D3FBFBA2FC5
:1025D000A92F982F8827820F911DA11DB11DBC0125
:1025E000CD0142E0660F771F881F991F4A95D1F7EA
:1025F0000895FB0141505109460F571FE417F50795
:1026000078F4208130E0322F22276181260F311D9E
:10261000820F931F8217930708F401963296EECF2C
:10262000E417F50751F4208130E0322F2227820F82
:10263000931F8217930708F4019608950E94713141
:10264000DC01ED91FC910190F081E02D0994611580
:10265000710579F0FB0101900020E9F73197AF0196
:10266000461B570BDC01ED91FC910280F381E02DBC
:10267000099480E090E008954F925F926F927F926C
:10268000EF92FF920F931F93CF93DF93CDB7DEB7F7
:10269000A1970FB6F894DEBF0FBECDBF7C01FA0143
:1026A000CB0119A2223008F42AE08E010F5D1F4FE2
:1026B000422E512C612C712CBF01A30192010E946A
:1026C000BC2EF901CA01015011096A3014F4605D91
:1026D00001C0695CD8016C93232B242B252B61F757
:1026E000B801C7010E942713A1960FB6F894DEBF68
:1026F0000FBECDBFDF91CF911F910F91FF90EF9053
:102700007F906F905F904F9008958F929F92AF92BD
:10271000BF92CF92DF92EF92FF920F931F93CF93CE
:10272000DF937C018B016C0182E0C80ED11C470154
:10273000E5E08E0E911CC0E0D0E0F60141916F0102
:1027400050E060E070E02AE0C8010E943C135C01A8
:102750006EE2C8010E9420138A0D9B1DC80FD91F6D
:10276000C814D90451F7F701458150E060E070E0EA
:102770002AE0C8010E943C138C0F9D1FDF91CF916E
:102780001F910F91FF90EF90DF90CF90BF90AF908F
:102790009F908F900895DC0190E020E030E08AE087
:1027A000FB014191BF01442309F150ED540F5A3010
:1027B00088F4829FF001839FF00D11249F01205324
:1027C0003109240F311D47FD3A952F3F310541F363
:1027D00038F312C04E3281F4933071F0FD01E90FED
:1027E000F11D22839F5F20E030E0DACF933021F4A7
:1027F00015962C9381E0089580E008951F920F9222
:102800000FB60F9211242F933F934F935F936F93C3
:102810007F938F939F93AF93BF93EF93FF9386E83C
:1028200094E00E944012FF91EF91BF91AF919F9170
:102830008F917F916F915F914F913F912F910F9069
:102840000FBE0F901F9018951F920F920FB60F9208
:1028500011242F938F939F93EF93FF93E09196040E
:10286000F09197048081E0919C04F0919D0482FD99
:1028700012C0908180919F048F5F8F732091A0047C
:10288000821751F0E0919F04F0E0EA57FB4F958FDB
:1028900080939F0401C08081FF91EF919F918F9160
:1028A0002F910F900FBE0F901F901895833081F0DD
:1028B00028F4813099F08230A1F008958730A9F092
:1028C0008830B9F08430D1F4809180008F7D03C0CE
:1028D000809180008F7780938000089584B58F77F2
:1028E00002C084B58F7D84BD08958091B0008F773C
:1028F00003C08091B0008F7D8093B00008951F9336
:10290000CF93DF93282F30E0F901ED5BFC4F8491EA
:10291000F901E559FC4FD491F901E95AFC4FC491F2
:10292000CC23C9F0162F81110E945614EC2FF0E031
:10293000EE0FFF1FE15DFC4FA591B4918FB7F894A6
:10294000111105C09C91ED2FE095E92302C0EC9197
:10295000ED2BEC938FBFDF91CF911F910895CF9313
:10296000DF9390E0FC01E559FC4F2491FC01E95A0A
:10297000FC4F8491882361F190E0880F991FFC013E
:10298000EB5DFC4FC591D491FC01E15DFC4FA5913D
:10299000B491611109C09FB7F89488812095822372
:1029A0008883EC912E230BC0623061F49FB7F894BA
:1029B0003881822F809583238883EC912E2B2C9352
:1029C0009FBF06C08FB7F894E8812E2B28838FBF56
:1029D000DF91CF9108958E3008F08E50877020914E
:1029E000000190E4299F90011124822B80937C00A8
:1029F00080917A00806480937A0080917A0086FDCD
:102A0000FCCF809178002091790090E0922B08957E
:102A10008F929F92AF92BF92CF92DF92EF92FF92EE
:102A20006B017C010E94D4124B015C01C114D104E2
:102A3000E104F104F1F00E94D412DC01CB01881909
:102A40009909AA09BB09883E9340A105B10570F315
:102A500021E0C21AD108E108F10888EE880E83E06F
:102A6000981EA11CB11CC114D104E104F10419F792
:102A7000DDCFFF90EF90DF90CF90BF90AF909F9011
:102A80008F9008952FB7F8946091B6027091B702B5
:102A90008091B8029091B9022FBF08951F920F92B2
:102AA0000FB60F9211242F933F938F939F93AF9361
:102AB000BF938091B6029091B702A091B802B091F5
:102AC000B9023091B50223E0230F2D3720F401968F
:102AD000A11DB11D05C026E8230F0296A11DB11D41
:102AE0002093B5028093B6029093B702A093B802E8
:102AF000B093B9028091BA029091BB02A091BC023E
:102B0000B091BD020196A11DB11D8093BA029093B0
:102B1000BB02A093BC02B093BD02BF91AF919F9145
:102B20008F913F912F910F900FBE0F901F9018958E
:102B3000A6EAB3E025E014969C91149798130DC073
:102B400095E0899FF0011124EA55FC4F8481149689
:102B50008C931382128214820895992331F0299F55
:102B6000D0011124AA55BC4FE6CF08950F931F93AF
:102B7000CF93DF938C01EB0160E08AE00E947F1429
:102B80008AE38EBD0DB407FEFDCF0C0F1D1FC017CD
:102B9000D10739F01EBC0DB407FEFDCF8EB5899369
:102BA000F6CF61E08AE0DF91CF911F910F910C94F5
:102BB0007F140F931F93CF93DF931F92CDB7DEB790
:102BC000182F062F60E08AE049830E947F14802F2F
:102BD0008F71812B8EBD49810DB407FEFDCF4EBD97
:102BE0000DB407FEFDCF61E08AE00F90DF91CF9139
:102BF0001F910F910C947F141F93CF93DF93182F85
:102C00001076C12FD0E02091020130E0C217D30727
:102C100089F043E06FE180EA0E94D915AE0185E0BA
:102C2000559547958A95E1F76FE180E80E94D9159F
:102C300010930201DF91CF911F9108951F93CF93BD
:102C4000DF9300D0CDB7DEB7182F69837A830E9457
:102C5000FC154981612F80E40E94D91561E0610F64
:102C60007A81472F80E40F900F90DF91CF911F91D1
:102C70000C94D9151F93CF93DF931F92CDB7DEB776
:102C8000182F69830E94FC154981612F80E40F9001
:102C9000DF91CF911F910C94D915CF93DF93C82F5B
:102CA000D62F60E08AE00E947F148D2F8F71C82B91
:102CB000CEBD0DB407FEFDCF1EBC0DB407FEFDCF8B
:102CC000D7FD08C061E08AE00E947F148EB5DF91D5
:102CD000CF9108951EBC0DB407FEFDCFF3CFCF9367
:102CE000DF931F92CDB7DEB7682F69830E94FC1572
:102CF000698180E00F90DF91CF910C944D16CF93B6
:102D0000DF93EB01682F84ED0E943A16BE0186ED39
:102D10000E941E16CFE0D0E08AEE0E946F1680FF60
:102D200008C06AE070E080E090E00E9408152197FA
:102D300099F7DF91CF910895CF93C62FBC0182E020
:102D40000E941E1660E08AE00E947F148AE78EBD12
:102D50000DB407FEFDCFCEBD0DB407FEFDCF61E083
:102D60008AE0CF910C947F14BC0180E00E941E1673
:102D700060E08AE00E947F148AE38EBD0DB407FEF6
:102D8000FDCF1EBC0DB407FEFDCF61E08AE00E94BE
:102D90007F148EB50895CF92DF92EF92FF920F933A
:102DA0001F93CF93DF936C018B014130510579F470
:102DB000CB010E94B416682FC601DF91CF911F91FD
:102DC0000F91FF90EF90DF90CF900C949C16EA014A
:102DD000C60FD71F7E0181E0E81AF10880E10E944A
:102DE0001E16B60184E10E941E160115184048F413
:102DF000E11488E0F80628F07E0181E0E81A88E016
:102E0000F80AB70182E10E941E1640E16FE180EAF4
:102E10000E94D91540E26FE180E80E94D9156FE168
:102E200080E00E944D1685FF07C061E070E080E001
:102E300090E00E940815F3CFDF91CF911F910F9181
:102E4000FF90EF90DF90CF900895CF92DF92EF92B6
:102E5000FF920F931F93CF93DF938C016091A60392
:102E60007091A7036150784EC12C98E1D92EE6EA03
:102E7000F3E080E0C0E0D0E045E09481992349F0A0
:102E8000499F900111242A553C4FD9012D913C9125
:102E900001C09B01E080F1802E193F090280F3817F
:102EA000E02D2E1B3F0B2017310739F4B5E08B9F27
:102EB000E0011124CA55DC4F49C00217130748F43A
:102EC0002C153D0530F4489FE0011124CA55DC4F14
:102ED0006901911107C02097C9F5C6EAD3E085E0E2
:102EE000D82E1EC0499FF0011124EA55FC4F892FAE
:102EF000C4CFEA80FB8028813981E20EF31ED89E80
:102F0000E0011124CA55DC4F68817981E616F70685
:102F100039F04A815B81C7010E94CB16F982E882B1
:102F20008C818111E6CF2091A6033091A70388817F
:102F30009981281B390B8A819B81281B390B2150D1
:102F4000384E2017310710F480E01AC091E0EBEA08
:102F5000F3E022813381232B29F035969F5F99324C
:102F6000C1F7F2CF4A815B8128813981240F351F57
:102F700031832083138302838C8184839C83892FF4
:102F8000DF91CF911F910F91FF90EF90DF90CF9045
:102F900008950F931F93DB01E42FA80190E0EF3F0A
:102FA000F9F065E0E69FF0011124EA55FC4F02C0FC
:102FB000E6E7F4E00190F081E02D2E0F3F1F65E081
:102FC000689FF001699FF00D1124EA55FC4F808144
:102FD0009181B9018A0F9B1F1F910F910C94CB1601
:102FE000E0917604F0917704E20FF31FE11568E0B9
:102FF000F607F0F29F012F5F3740E1CFCF92DF92CB
:10300000EF92FF920F931F93CF93DF937B018A017F
:10301000690125E0829FC0011124EC01CA55DC4FF3
:10302000688179816E0D7F1D82E00E941E160A80E4
:10303000DB81C02DCE19DF09CC16DD0608F4E601D0
:1030400060E08AE00E947F148AE78EBD0DB407FE1F
:10305000FDCFC8018C0F9D1F0817190741F0F8011B
:1030600021918F012EBD0DB407FEFDCFF5CF61E09C
:103070008AE00E947F14CE01DF91CF911F910F91C2
:10308000FF90EF90DF90CF900895EF92FF920F9313
:103090001F93CF93DF938B017A018F3FD1F025E00F
:1030A000829FE0011124CA55DC4F02C0C6E7D4E07C
:1030B00088819981B801680F791F80E00E941E16EF
:1030C0008A819B81801B910BE816F90690F4C70159
:1030D00010C08091760490917704860F971F811518
:1030E00028E0920718F3BC016F5F7740C6E7D4E091
:1030F000E4CFDF91CF911F910F91FF90EF90089552
:103100008823A1F090917304992381F08F3F29F4D3
:103110008091780490917904089595E0899FF00159
:103120001124EA55FC4F82819381089580E090E05C
:103130000895EF92FF920F931F93CF93DF938091A7
:10314000610290E0982F882720916202820F911DE2
:103150007C0124E1E21AF10848E050E06BE672E0FD
:103160000E970E94F912C0917F02C695C695CC7346
:10317000D0E0AE0163E772E00E94F9128C01CE1537
:10318000DF0508F04CC0A7014C1B5D0BBE016E5D56
:103190007F4F809150020E944518EC01219760E01A
:1031A0008AE00E947F148AE38EBD0DB407FEFDCF36
:1031B000A80160E070E06C177D07C8F41EBC0DB478
:1031C00007FEFDCF2EB530E0322F22271EBC0DB4F6
:1031D00007FEFDCF8EB5280F311D420F531F42173A
:1031E000530710F44F5F5F4F6E5F7F4FE4CF8A014C
:1031F0006C177D0781F41EBC0DB407FEFDCF8EB5A4
:1032000090E0982F88278A01080F191F08171907BF
:1032100010F40F5F1F4F61E08AE00E947F140115D8
:10322000110519F0902F812F02C08FEF9FEFDF91D2
:10323000CF911F910F91FF90EF90089544E150E0DE
:103240006FE572E080E090E00E94F912009721F0B3
:1032500098278927982708958FEF9FEF0895CF9299
:10326000DF92EF92FF92CF93DF93B09176058823A0
:1032700011F0AB2F01C0A0E08091770590E0880F9E
:10328000991F875C9C4FC0907C05D0907D05E09095
:103290007E05F0907F0520E030E0FC01C591D491DF
:1032A000E881EB23A90160E070E0EA130CC02F5F16
:1032B0003F4F4C155D056E057F0578F33FEF2FEF0F
:1032C0008FEF9FEF03C0322F252FCB01632F722F7B
:1032D000DF91CF91FF90EF90DF90CF900895CF9244
:1032E000DF92EF92FF92CF93DF93EC010E944215A1
:1032F0006B017C018091860590918705DC01ED9141
:10330000FC910084F185E02D0995892B79F40E94C8
:103310004215AB01BC014C195D096E097F094839A2
:103320005A436105710530F380E00DC08091860538
:1033300090918705DC01ED91FC910284F385E02DED
:103340000995888381E0DF91CF91FF90EF90DF9026
:10335000CF9008958F929F92AF92BF92CF92DF92BB
:10336000EF92FF920F931F93CF93DF9300D000D083
:1033700000D0CDB7DEB78C016B017A0159010E94F4
:103380004215DC01CB0186509F4FAF4FBF4F80935A
:10339000810490938204A0938304B09384041092D8
:1033A00077041092760410927904109278048DECD0
:1033B000E6EAF3E0DF011D928A95E9F781E098E003
:1033C0009093A7038093A60361E08AE00E94AF1464
:1033D00061E08AE00E947F1461E08BE00E94AF14FC
:1033E00061E08DE00E94AF1460E08CE00E94AF14B9
:1033F00061E08AE00E94AF1461E08AE00E947F14DD
:1034000060E08BE00E947F1460E08DE00E947F14FA
:1034100080E58CBD8DB581608DBD4FEF60E08FEF95
:103420000E94D91562E070E080E090E00E940815EB
:1034300062E370E080E090E00E940815109275044D
:103440001092740420E1822E912C6DE180E00E94A4
:103450004D1681110BC0B1E08B1A910839F06AE06A
:1034600070E080E090E00E940815EFCF60E070E02F
:1034700088E00E941E1660E070E08CE00E941E163C
:103480006FEF77E08AE00E941E1661EB88E30E94EE
:103490003A166FE370E388E20E941E1669EF77EF39
:1034A00080E30E941E166DE070E080EC0E941E1604
:1034B00042E362EC80E80E94D91562E17CE086EC90
:1034C0000E941E1662E184EC0E943A166CED75E0D3
:1034D0008AEC0E941E1660912C0584EE0E943A161A
:1034E00060912D0585EE0E943A1660912E0582EEC0
:1034F0000E943A1660912F0583EE0E943A16609161
:10350000300580EE0E943A166091310581EE0E94EE
:103510003A1660E071E080E10E947F168FE10E9420
:10352000FC1540EC6BE180E80E94D91544E06FE1A6
:1035300080E80E94D91566E774E084E10E947F1656
:1035400082E70E946F168F3F09F0BAC01092730491
:1035500080912C0580937B0480912D0580937C04C1
:1035600080912E0580937D0480912F0580937E04A9
:103570008091300580937F04809131058093800491
:1035800080E0E82FF0E0EE0FFF1FE356FC4F1182C2
:1035900010828F5F8430A9F780E09EE1989FF00150
:1035A0001124EB5DFC4F118E8F5F8430B9F780934F
:1035B000A50380E094E0909324038093230310926A
:1035C00022039BE080912203883068F4989FF001E9
:1035D0001124E653FD4F10821182128213828F5FF5
:1035E00080932203EFCFF50192805381B4819581BE
:1035F000F701A2818381B4804581F601C280D38026
:10360000E480F580F801248130E0322F22276581A3
:10361000262B322723273227628170E0762F6627F8
:103620001381612B7627672776277093C7026093F3
:10363000C6023093C9022093C802282F30E03A2BEB
:103640003827232732273093C3022093C202242F26
:1036500030E03B293427232732273093C5022093BB
:10366000C402252F30E0392935272327322730930C
:10367000BF022093BE02892F90E09B2B98278927B9
:1036800098279093C1028093C002C0922505D092E2
:103690002605E0922705F092280526960FB6F894A5
:1036A000DEBF0FBECDBFDF91CF911F910F91FF9075
:1036B000EF90DF90CF90BF90AF909F908F90089544
:1036C0008093730445CFCF93DF93E1E5F3E08491DA
:1036D000E9E7F3E0D491E5E6F3E0C491CC2391F07F
:1036E00081110E945614EC2FF0E0EE0FFF1FE75CF3
:1036F000FC4FA591B491EC91ED2381E090E021F491
:1037000080E002C080E090E0DF91CF910895CF92F9
:10371000DF92EF92FF92CF93DF93AB01BC0177FF73
:103720001DC06A017B016DE286E894E00E942013CF
:10373000EC0144275527BA014C195D096E097F0930
:103740002AE086E894E00E943C138C0F9D1FDF91D5
:10375000CF91FF90EF90DF90CF9008952AE086E818
:1037600094E0DF91CF91FF90EF90DF90CF900C9499
:103770003C135F926F927F928F929F92AF92BF9213
:10378000CF92DF92EF92FF920F931F93CF93DF932D
:103790001F92CDB7DEB74C0188E895E00E946F1903
:1037A000882309F441C070908805198201E010E077
:1037B000A12CB12CC12CD12C7601C394CE01019641
:1037C0000E946F19882381F10F5F1F4F8981F801D3
:1037D000EE57FA4F8583282F2F7730E02C9DA001DC
:1037E0002D9D500D3C9D500D1124A40EB51E37E0AB
:1037F000CC0CDD1CEE1CFF1C3A95D1F787FF17C0DF
:1038000005301105D9F68FEF9FEF90932206809334
:1038100021068091860590918705DC01ED91FC9150
:103820000488F589E02D099580E090E07CC0872D23
:10383000807F55245394803309F0512C8FEF800FF3
:10384000F4018083552021F1C80188579A4F0E94C6
:103850006F19882349F3C80187579A4F0E946F193F
:10386000882311F30E5F1F4FD401EC91F0E0EE5767
:10387000FA4FE780F12CFE2CEE248085E80EF11C37
:103880008091880581FF08C0B2E0EB0EF11C04C0F6
:1038900080E0E12CF12C01C082E0C82ED12CC01AAE
:1038A000D10A9EEF692E77247A94C601800F911F6A
:1038B0008A159B0568F5CE0101960E946F19882331
:1038C00009F4B2CF80911F06909120060097A9F0CD
:1038D000552099F0F4012081A301421B51099A015E
:1038E000200F311FE216F30640F4DC01ED91FC914C
:1038F0000190F081E02D698109950038110528F4C7
:103900008981F801EE57FA4F86830F5F1F4FCDCFA5
:1039100080911F0690912006892B21F40138110512
:1039200008F082CFC8010F90DF91CF911F910F91C6
:10393000FF90EF90DF90CF90BF90AF909F908F90CF
:103940007F906F905F9008954F925F926F927F92F9
:103950008F929F92AF92BF92CF92DF92EF92FF929F
:103960006B017C01B42E9B01AC010E94663188235F
:1039700019F067EB71E027C026013701E89477F86A
:103980002FEF3FEF4FE75FE7C301B2010E946631BF
:1039900081110DC02FEF3FEF4FE75FE7C301B20189
:1039A0000E949C2F18161CF46BEB71E00CC02FEFDB
:1039B0003FEF4FE75FE4C701B6010E94F4301816ED
:1039C00094F46FEB71E086E894E0FF90EF90DF9065
:1039D000CF90BF90AF909F908F907F906F905F90AF
:1039E0004F900C9427132FEF3FEF4FE75FECC70189
:1039F000B6010E949C2F87FDE4CF20E030E0A901B2
:103A0000C701B6010E949C2F87FF0BC06DE286E8BC
:103A100094E00E9420134C01F7FAF094F7F8F09428
:103A200002C0812C912CA12C60E070E080E09FE32B
:103A3000AB1441F020E030E040E251E40E94A12FBD
:103A4000A394F6CF9B01AC01C701B6010E94302FB1
:103A50002B013C010E9413306B017C010E9442301B
:103A60009B01AC01C301B2010E942F2F2B013C012D
:103A70002AE0B701A60186E894E00E943C137C018D
:103A8000E80CF91CBB2039F06EE286E894E00E9455
:103A90002013E80EF91EDB2CDD2031F120E030E0B0
:103AA00040E251E4C301B2010E94F9302B013C0114
:103AB0000E9413304B01A12CB12C2AE0B501A401C6
:103AC00086E894E00E943C13E80EF91EC501B4019B
:103AD0000E9442309B01AC01C301B2010E942F2F12
:103AE0002B013C01DA94D8CFC701FF90EF90DF9013
:103AF000CF90BF90AF909F908F907F906F905F908E
:103B00004F900895CF92DF92EF92FF920F931F9301
:103B1000CF93DF93CDB7DEB7C054D1400FB6F89442
:103B2000DEBF0FBECDBF0E944215009178051091F7
:103B3000790520917A0530917B056B017C01C01AD3
:103B4000D10AE20AF30A40EDC41647E0D406E104C4
:103B5000F10418F480918005CAC0609378057093D1
:103B6000790580937A0590937B05109273051092E6
:103B70007205109271051092700510926F0562E047
:103B8000809174050E94AF1461E070E080E090E0E5
:103B90000E94081561E0809174050E94AF1460E0F6
:103BA000809174050E947F14809175058551823043
:103BB00028F48BE291E10197F1F706C064E170E02F
:103BC00080E090E00E94081562E0809174050E94F8
:103BD000AF148091810590E08230910538F0880F14
:103BE000991F880F991F05970197F1F7F89480E0C6
:103BF0000E942F196F3F7F4F8F4F9F4F21F41092DC
:103C00008005789441C081E00E942F196F3F7F4F5B
:103C10008F4F9F4FA1F38E010F5F1F4F6E012FEB50
:103C2000C21A2EEFD20A780180E00E942F19F70104
:103C3000608371838283938381E00E942F19F7014F
:103C40006483758386839783F8E0EF0EF11CEC1490
:103C5000FD0451F7789420E030E0F8014081518173
:103C600062817381C480D580E680F7804F3FFFEF8B
:103C70005F076F077F0731F08FEFC816D806E80699
:103C8000F80621F41092800580E031C0F90183E04C
:103C9000F595E7958A95E1F7E159FA4F8081880F0C
:103CA0004C155D056E057F0508F4816080832F5FEC
:103CB0003F4F085F1F4F2832310579F62091730579
:103CC00030E040916F058091700590E0840F911D68
:103CD00040917105840F911D40917205840F911DD3
:103CE00099272817390771F681E080938005C05C19
:103CF000DE4F0FB6F894DEBF0FBECDBFDF91CF9180
:103D00001F910F91FF90EF90DF90CF900895CF9388
:103D1000DF93DC014E5F5F4FFC019F012A1B3B0BD1
:103D20009191992339F0EB01C40FD51F98834F5F10
:103D30005F4FF3CFCA01821B930B680F791FFB0102
:103D40003297308331962083CA01DF91CF91089555
:103D5000CF92DF92EF92FF920F931F93CF93DF9357
:103D600000D000D0CDB7DEB7FA0130E09E2F9F77AC
:103D7000EE0FEF2FEE1FFF0BF195309709F09068D3
:103D800021E0230FA1E0B0E0AC0FBD1FA30FB11DD8
:103D90009C93309711F0322FE9CF30E0DB01A21B6A
:103DA000B30B14968C93CE0101966C0180E090E0E9
:103DB0008217930764F4F60111916F017C01E21AF6
:103DC000F30AE60EF71EF70115830196F1CF8091F5
:103DD0008605909187052F5F3F4F8901040F151FBE
:103DE000FC0120813181F90122813381A801BD01CB
:103DF000F90109957C010E94421560930A067093AF
:103E00000B0680930C0690930D0681E0E016F106F8
:103E100009F080E00F900F900F900F90DF91CF91FD
:103E20001F910F91FF90EF90DF90CF9008958091B8
:103E3000860590918705009759F1DC01ED91FC9181
:103E40000688F789E02D0995811124C0809121060B
:103E500090912206892BE1F48DEF9FEF909322063B
:103E6000809321068091860590918705DC01ED9174
:103E7000FC910680F781E02D09958091860590914F
:103E80008705DC01ED91FC910488F589E02D099509
:103E900080E0089581E00895CF93DF93FC010190C5
:103EA0000020E9F79F01281B390B285F3F4F21387D
:103EB000310570F5EC010E94171F882349F18091AC
:103EC000080690910906019611F481E090E0909324
:103ED0000906809308068091080690910906909340
:103EE0008D0580938E0547E050E068E875E0CE01CF
:103EF0000E94871EFC01EE57FA4F1682AC01445017
:103F0000510968E875E082E8DF91CF910C94A81E12
:103F100080E0DF91CF910895BC0186E894E00C9495
:103F200027130F931F93CF93DF938C01C0E0D0E052
:103F3000F801EC0FFD1F6491662371F0E091860497
:103F4000F09187040190F081E02D86E894E00995D6
:103F5000892B11F02196ECCFCE01DF91CF911F91EB
:103F60000F910895EF92FF920F931F93CF93DF93DA
:103F70007C018B01EB0109900020E9F72197C61B1A
:103F8000D70B0E94171F8823B1F1F7010190002081
:103F9000E9F73197EE19FF09CE010796E80FF91FEF
:103FA000E138F10540F545E050E068E875E0C7010B
:103FB0000E94871EF80120E030E02C173D0759F0E1
:103FC0004191D901A80FB91FAE57BA4F16964C931D
:103FD0002F5F3F4FF2CF25503109A901480F591FDC
:103FE00068E875E080E3DF91CF911F910F91FF901A
:103FF000EF900C94A81E80E0DF91CF911F910F915C
:10400000FF90EF9008956BED71E086E894E00C94DA
:104010002713CF93DF93BC0186E894E00E94271317
:10402000EC010E9403208C0F9D1FDF91CF9108951A
:10403000CF93DF930E94911FEC010E9403208C0F0D
:104040009D1FDF91CF910895FC0182819381A4810E
:10405000B5818093170690931806A0931906B09324
:104060001A068BE597E090931E0680931D0610922A
:104070001C0610921B0682E895E00895CF93DF930B
:1040800066E874E00E948513EC010E9403208C0F07
:104090009D1FDF91CF910895CF93DF93CDB7DEB70A
:1040A000C854D1090FB6F894DEBF0FBECDBF7894C7
:1040B00084B5826084BD84B5816084BD85B582602D
:1040C00085BD85B5816085BD80916E0081608093DE
:1040D0006E00109281008091810082608093810047
:1040E0008091810081608093810080918000816057
:1040F000809380008091B10084608093B1008091B2
:10410000B00081608093B00080917A0084608093D9
:104110007A0080917A00826080937A0080917A00A0
:10412000816080937A0080917A00806880937A0021
:104130001092C100E0919604F091970482E0808390
:10414000E0919204F09193041082E0919404F09134
:10415000950480E1808310929E04E0919A04F0918E
:104160009B0486E08083E0919804F091990480811B
:1041700080618083E0919804F09199048081886047
:104180008083E0919804F091990480818068808315
:10419000E0919804F091990480818F7D80838AEA70
:1041A00091E00E94911F82E691E00E9409208AE935
:1041B00091E00E9418200FB6F894A89580916000B5
:1041C000886180936000109260000FBE62E08FE013
:1041D0000E94AF1462E080E10E94AF1462E081E1CE
:1041E0000E94AF1462E082E10E94AF1462E083E1BA
:1041F0000E94AF1462E084E10E94AF1462E08EE09E
:104200000E94AF1461E083E00E94AF1461E084E09B
:104210000E94AF1461E085E00E94AF1461E086E087
:104220000E94AF1461E087E00E94AF1461E088E073
:104230000E94AF1461E082E00E94AF1481E080939D
:10424000000161E082E00E947F1480E090E00E9423
:10425000962E90912905891759F00E94631B21E041
:10426000892B09F420E020930101211113C0B9C06A
:1042700019E2E12E15E0F12E00E010E0C8010E94E5
:10428000962ED7018D937D010F5F1F4F06341105C8
:10429000A9F7E3CF0AE511E01A8309838091460567
:1042A00090914705A0914805B09149058B839C8367
:1042B000AD83BE831B8F0A8F80914005909141058D
:1042C000A0914205B09143058C8F9D8FAE8FBF8F1B
:1042D0001DA70CA780913A0590913B05A0913C0544
:1042E000B0913D058EA79FA7A8ABB9AB1FAF0EAF8E
:1042F0008091340590913505A0913605B091370530
:1043000024968CAF9DAFAEAFBFAF24979E012F5FB9
:104310003F4FAE01465E5F4FBE01645D7F4FCE01F1
:10432000CE960E94AA198EE891E00E94911F3091CA
:10433000C6022091C7029091C8028091C9021A83D7
:1043400009833B832C839D838E83CE0101960E943B
:104350003E2083E296E090938705809386051A833A
:10436000098380914C0590914D05A0914E05B09127
:104370004F058B839C83AD83BE83CE0101960E9443
:10438000242081E391E1909314068093130681E841
:1043900091E00E9418208091680590916905A09194
:1043A0006A05B0916B05B095A095909581959F4F4A
:1043B000AF4FBF4F8093E6019093E701A093E801D0
:1043C000B093E90180912A05882379F099E288E188
:1043D0000FB6F894A895809360000FBE909360008C
:1043E00004C082E791E00E94182062E089E00E9408
:1043F000AF14F0906E0580916C0599E09093740570
:1044000080937505E4E7F3E0E491E0937605E0E658
:10441000F3E0E491E093770562E089E00E94AF1455
:104420000E94421528EE33E0F29E8001F39E100DAB
:104430001124012E000C220B330BDC01CB01801B5D
:10444000910BA20BB30B8093780590937905A09301
:104450007A05B0937B0587E38093810560ED77E073
:1044600080E090E00E940815FE0131967F014E0128
:10447000FCE28F0E911C6E012AE1C20ED11C00E0FD
:1044800010E0BAE5AB2EB1E0BB2E86E894E00E94C6
:104490002A12892B09F4DEC186E894E00E940812F2
:1044A0008A3051F08D3009F4CAC1F701E00FF11FD5
:1044B00080830F5F1F4FC3C1FFAEEEAEAE01425C03
:1044C0005F4F66E671E0C7010E94B42BBC01C401D6
:1044D0000E94B4318401F40101900020E9F7319782
:1044E000E819F909C801881999098E179F0758F426
:1044F000D8018C91082E000C990B0E947631F8019E
:1045000081938F01E8CF1CA51F3329F48EEF91E032
:104510000E94182092C1173551F4EEADFFAD81E035
:1045200091819E3409F080E080932A0586C11D3474
:1045300011F58DA58134C9F56EAD7FADC6010E9420
:10454000B43168E671E0C6010E94AF2B0CE215E0C1
:10455000009709F472C140E150E060E070E00E9411
:104560004F2AD8016D938D0168E671E080E090E0FC
:104570000E94AF2BEDCF193429F46EAD7FAD82E3ED
:1045800095E009C0143451F48DA58E34C1F56EAD9B
:104590007FAD88E395E00E94CB134FC1173469F4D7
:1045A0006EAD7FAD8EE395E0F6CF833509F014C193
:1045B0006EAD7FAD84E495E0EECF133549F48DA563
:1045C000863509F009C16EAD7FAD8AE495E0E3CF91
:1045D000133429F46EAD7FAD80E595E006C0153546
:1045E00039F46EAD7FAD86E595E00E94B43125C10A
:1045F0001035A9F46EAD7FAD8FE595E0F6CF8C3424
:1046000009F0EAC08EAD9FAD0E947F2B60936805D4
:104610007093690580936A0590936B050EC11F34F2
:1046200009F0DAC089EF91E00E94911F60912A059C
:1046300070E080E090E00E94871B0E94032084EFDE
:1046400091E00E94911F60916C0570916D05072E9D
:10465000000C880B990B0E94871B82EF91E00E944F
:10466000911F40916E0550E060E070E02AE086E81E
:1046700094E00E943C130E9403208DEE91E00E9482
:10468000911F00E010E0F801E75DFA4F438150E030
:1046900060E070E020E186E894E00E943C13053081
:1046A000110511F06AE301C06AE086E894E00E9417
:1046B00020130F5F1F4F0630110529F788EE91E098
:1046C0000E94911FBB8EAA8E809134059091350572
:1046D000A0913605B09137058C8F9D8FAE8FBF8F1F
:1046E000C6010E943E2083EE91E00E94911FBB8E86
:1046F000AA8E80913A0590913B05A0913C05B0911E
:104700003D058C8F9D8FAE8FBF8FC6010E943E20CE
:104710008EED91E00E94911FBB8EAA8E8091400584
:1047200090914105A0914205B09143058C8F9D8FDA
:10473000AE8FBF8FC6010E943E2089ED91E00E949E
:10474000911FBB8EAA8E8091460590914705A0913E
:104750004805B09149058C8F9D8FAE8FBF8FC601E4
:104760000E943E2084ED91E00E94911FBB8EAA8E94
:1047700080914C0590914D05A0914E05B0914F054B
:104780008C8F9D8FAE8FBF8FC6010E943E208FEC15
:1047900091E00E94911F80E595E00E9409208AEC3B
:1047A00091E00E94911F86E595E00E94092085EC2A
:1047B00091E00E94911F8FE595E00E94092080EC16
:1047C00091E00E94911F6091680570916905809148
:1047D0006A0590916B052DC06AE671E0C4010E94E4
:1047E000AB31892B91F4A9E26A2EA5E07A2E00E084
:1047F00010E0F30161913F01C8010E949E2E0F5FFE
:104800001F4F06341105A9F718C01D34B1F48DA54A
:10481000853499F480915D0690915E06009711F4BD
:1048200083E696E0B601681B790B072E000C880B17
:10483000990B0E94871B0E94032000E010E0F70103
:10484000E00FF11F10826AE070E080E090E00E94CB
:1048500008151BCE8091EA01882329F00E94631B72
:10486000019709F422C20E9442150091E6011091BD
:10487000E7012091E8013091E901DC01CB01801BC7
:10488000910BA20BB30B0091680510916905209163
:104890006A0530916B05081719072A073B0748F08E
:1048A0008091EA018111B2C00E94631B892B09F03B
:1048B000ADC080E595E00E948C1F81E293E00E94EC
:1048C000911F0E94821D882309F408C280917505FA
:1048D0008B3008F403C28D3008F0EAC160916F0597
:1048E00070E080E090E00E9444302B013C01809118
:1048F0007005682F70E080E090E00E9444302DEC5D
:104900003CEC4CEC5DE30E94F9309B01AC01C3012F
:10491000B2010E94302F6093E2017093E301809313
:10492000E4019093E5010E94821D882309F416C2D8
:10493000809175058C3009F4EEC108F0D4C18B303C
:1049400009F00CC26091710570E080E090E00E9477
:1049500042302B013C011091720517FF0AC09B01E8
:10496000AC0160E070E080E89FEB0E942F2F2B01EC
:104970003C01812F8F70682F70E080E090E00E94F2
:1049800044302DEC3CEC4CEC5DE30E94F9309B0193
:10499000AC01C301B2010E94302F6093DE0170931D
:1049A000DF018093E0019093E1018AE193E00E94AE
:1049B000911F6091DE017091DF018091E001909183
:1049C000E10142E00E94A41C83E193E00E94911F58
:1049D0006091E2017091E3018091E4019091E50121
:1049E00040E00E94A41C109101011111BCC10E9461
:1049F000032081E08093EA010E9442156093E60162
:104A00007093E7018093E8019093E901809101019F
:104A1000882309F43CC10E94171F882309F437C179
:104A20000E9442151B012C0180910E0690910F06E9
:104A3000A0911006B0911106A2019101281B390B1B
:104A40004A0B5B0BDA01C90189399A43A105B1050B
:104A5000A8F480910A0690910B06A0910C06B091E3
:104A60000D06A2019101281B390B4A0B5B0BDA01E1
:104A7000C90189399A43A105B105C8F120911206EF
:104A80008091860590918705222371F02CEF3FEFEE
:104A90003093220620932106DC01ED91FC910488DD
:104AA000F589E02D0995F3C020EC2093880510923C
:104AB0008905DC01ED91FC910280F381E02D42E05B
:104AC00050E068E875E0099520920A0630920B06DE
:104AD00040920C0650920D0620920E0630920F0660
:104AE000409210065092110681E080931206809148
:104AF000860590918705DC01ED91FC910084F1859C
:104B0000E02D0995892B09F4C2C0C7010E94B91B89
:104B10009C01892B09F4B9C020920E0630920F0631
:104B2000409210065092110680918805807F803354
:104B300009F08FC08091130690911406892B09F417
:104B4000A6C0A980B12CF501EE57FA4F078110E0FD
:104B5000102F00278085080F111DF501E657FA4F29
:104B60003F01B50165577A4FA801CF0128962FAFB5
:104B7000289729963FAF29970E948731B8016A0D7F
:104B80007B1DFB01EE57FA4F1086809188058670D9
:104B900027968FAF2797A0911306B09114062896F9
:104BA0002FAD289729963FAD2997823009F043C051
:104BB000818590E0982F88274285FC01E40FF11D44
:104BC0002696FFAFEEAF26974BEF5FEF4A195B09D2
:104BD000401B510B420F531F63577A4FC301FD0116
:104BE000099580E48093880527962FAD2797209319
:104BF000890526963FAD269730938A0525964FADB9
:104C0000259740938B058091860590918705DC015F
:104C1000ED91FC910280F381E02D44E050E068E8E2
:104C200075E0099520920A0630920B0640920C0618
:104C300050920D062CC04DEF5FEF4A195B09401BE7
:104C4000510B420F531F65577A4FC301FD01099560
:104C50001EC0803CA9F480ED8093880510928905E0
:104C60008091860590918705DC01ED91FC91028091
:104C7000F381E02D42E050E068E875E0099507C057
:104C8000803D29F41092120602C00E94171F8091E5
:104C90002A05882309F0A8956AE070E080E090E09A
:104CA0000E9408150E94CA12EACB1092EA01DBCDDD
:104CB0008551823098F460916F0570E0762F6627F9
:104CC00080917005682B80E090E00E9442302DECCE
:104CD0003CEC4CEC5DE30E94F9301DCE60E070E0EE
:104CE00080EC9FE718CE85518230C0F51091710598
:104CF000612F6F7770E0762F662780917205682BA1
:104D000080E090E00E9442302DEC3CEC4CEC5DE306
:104D10000E94F9301FC010917105612F70E080E092
:104D200090E00E9442302B013C01809172058F700F
:104D3000682F70E080E090E00E9444302DEC3CEC65
:104D40004CEC5DE30E94F9309B01AC01C301B20160
:104D50000E94302F17FF21CE90581FCE60E070E0E8
:104D600080EC9FE71ACE0E946C040E94171F8111ED
:104D70000DC160911B0670911C0680918605909173
:104D8000870540911D0650911E06DC01ED91FC91B6
:104D90006115710521F00088F189E02D14C00684A9
:104DA000F785E02D2AE531E03A8329834090170604
:104DB000509018066090190670901A064B825C821B
:104DC0006D827E82B70109958130910509F0D7C0C7
:104DD000909309068093080687E0E3E0F1E0D701AD
:104DE00001900D928A95E1F7F701ADE8B5E0CE01AB
:104DF000089621912D93E817F907D9F786E595E0F4
:104E0000892B31F08FE595E0892B21F082EC03C0EE
:104E100082E001C082E880939405109295058FE0AE
:104E200080939605E0E5F5E001900020E9F7CF01D9
:104E3000805495408138910508F095C04FE050E0CE
:104E400068E875E080E595E00E94871EE6E5F5E0FC
:104E5000309741F101900020E9F7E80FF91FE5557F
:104E6000F540E138F10508F07EC0AC0168E875E076
:104E700086E595E00E94871EEFE5F5E0309791F01A
:104E800001900020E9F7E80FF91FEE55F540E138F1
:104E9000F10508F068C0AC0168E875E08FE595E0C1
:104EA0000E94871EAC014550510968E875E080E119
:104EB0000E94A81E0E94421560930A0670930B067A
:104EC00080930C0690930D0660930E0670930F0668
:104ED0008093100690931106809186059091870526
:104EE000DC01ED91FC910084F185E02D0995892B81
:104EF000C1F40E94421540900E0650900F0660903B
:104F0000100670901106DC01CB0184199509A609E1
:104F1000B70988399A43A105B105F0F28CEF9FEFEC
:104F20001EC0C6010E94B91B0497E9F480918B054D
:104F3000811114C00E94421560930E0670930F06F3
:104F4000809310069093110610921206109222067A
:104F500010922106112309F44ACD18C090E09093D5
:104F60002206809321068091860590918705DC01B9
:104F7000ED91FC910488F589E02D099538CD8EEFEF
:104F80009FEF909322068093210631CD6091DE0140
:104F90007091DF018091E0019091E101870122E0B1
:104FA00046E00E942F2A8C016C2D8FE691E00E9432
:104FB0001511B8010E94B21F6091E2017091E301E6
:104FC0008091E4019091E501870120E046E00E9494
:104FD0002F2A8C016C2D84E791E00E941511B801F5
:104FE0000E94B21F8FE00E94EB144AE0B7010E94BA
:104FF000DB2B6C2D89E791E00E941511B7010E940F
:10500000B21F8CE093E00E94911FC7010E948C1F89
:1050100080E10E94EB144AE0B7010E94DB2B6C2D6B
:105020008EE791E00E941511B7010E94B21F85E042
:1050300093E00E94911FC7010E948C1F81E10E9492
:10504000EB144AE0B7010E94DB2B6C2D83E891E062
:105050000E941511B7010E94B21F8EEF92E00E94CC
:10506000911FC7010E948C1F82E10E94EB144AE04D
:10507000B7010E94DB2B6C2D88E891E00E9415118E
:10508000B7010E94B21F87EF92E00E94911FC701F3
:105090000E948C1F83E10E94EB144AE0B7010E943A
:1050A000DB2B6C2D8DE891E00E941511B7010E9459
:1050B000B21F80EF92E00E94911FC7010E948C1FD7
:1050C00084E10E94EB144AE0B7010E94DB2B6C2DB7
:1050D00082E991E00E941511B7010E94B21F89EE8A
:1050E00092E00E94911FC7010E948C1F6C2D87E9DE
:1050F00091E00E9415110E944C1F6C2D8CE991E0EB
:105100000E9415110E944C1F6C2D81EA91E00E94B3
:1051100015110E944C1F6C2D86EA91E00E9415111A
:105120000E944C1F6C2D8BEA91E00E9415110E9489
:105130004C1F6C2D80EB91E00E9415110E944C1FBA
:1051400061E082E00E947F1464E670E080E090E01D
:105150000E94081560E082E00E947F1448CCFC01A8
:105160002381260F20934602A72FBB2792819A0FF7
:105170009093450231813093440240814093430231
:10518000E92FF0E0EA17FB0748F481E0830F8093F2
:105190004402811103C04F5F4093430230E0772700
:1051A0002617370788F49F5F9093450291110CC032
:1051B000809144028F5F80934402811105C08091E9
:1051C00043028F5F8093430208952091F60130914E
:1051D000F701BC01C90108960E94AF28E091F601D1
:1051E000F091F701A3E4B2E08C91808711968C9145
:1051F0001197818712968C911297828713968C91C2
:1052000083870895CF93DF93E1E3F6E08AE591E0A9
:10521000918380831282138214821582E6E8F4E07F
:105220001382128248EE53E060E070E044835583BD
:10523000668377832AE131E03183208325EC30E0F7
:105240003587248724EC30E03787268720EC30E050
:10525000318B208B21EC30E0338B228B22EC30E041
:10526000358B248B26EC30E0378B268B118E128EFB
:10527000138E148EE7E3F6E091838083128213820B
:1052800014821582EDE3F6E091838083128213820B
:1052900014821582E3E4F6E0918380831282138204
:1052A00014821582E3E2F5E09183808312821382F7
:1052B00014821582E9E4F6E09183808312821382DE
:1052C00014821582EFE4F6E09183808312821382C8
:1052D00014821582E5E5F6E09183808312821382C1
:1052E00014821582E3E2F6E013821282448355832E
:1052F0006683778328E331E0318320831586148623
:10530000E2E8F5E0138212822CE231E0318320835F
:1053100090931606809315061092170610921806A1
:105320001092190610921A062FEF3FEF30932206C3
:1053300020932106158214821092200610921F06D7
:105340001092140610921306AFE6B5E029E0159608
:105350002C93159726E116962C931697E4E7F3E025
:10536000E4911796EC931797E0E6F3E0E491189632
:10537000EC93189740E85EE360E070E01D964D9373
:105380005D936D937C935097C9E2D5E022E1288329
:10539000198221E02A8326E0E0E1F1E0ACE2B5E009
:1053A00001900D922A95E1F79A87898730EC3B8727
:1053B00028EA2C871D864DE04E87988B8F8744ED19
:1053C000498B4BE14A8B48E24B8B40EF4C8B9E8BD9
:1053D0008D8B3F8B288F198E4EEF4A8F9C8F8B8F32
:1053E0004FEF4D8F4E8F4F8F18A29AA389A33BA3E7
:1053F0002CA31DA284EB8EA386E0E3ECF1E0A0E5F4
:10540000B5E001900D928A95E1F789E0E9ECF1E0D1
:10541000A6E5B5E001900D928A95E1F789E0E2ED0D
:10542000F1E0AFE5B5E001900D928A95E1F788E8EB
:1054300093E1A0E0B0E08093680590936905A093A4
:105440006A05B0936B0586E190E090936D058093BB
:105450006C0582E080936E05DF91CF910895EF9205
:105460000F931F93CF93DF93E80147FD02C034E011
:1054700001C034E1E42F440FFF0BF7FF03C0F195A7
:10548000E195F109E32E022F2E2FAE010E941D2C73
:10549000CE01DF91CF911F910F91EF900895A6E07B
:1054A000B0E0E5E5FAE20C94E92E5C016B017A01CB
:1054B0006115710519F0DB018D939C93E114F104E2
:1054C00029F0C7010297839708F0DCC03501BFEFD0
:1054D0006B1A7B0AF5011081812F90E00E94A62BA8
:1054E000892B11F05301F2CF1D3249F43501F2E05E
:1054F0006F0E711CD50111961C9101E009C01B3281
:1055000031F43501B2E06B0E711CF501118100E040
:10551000E114F10409F4C4C0F0E1EF16F10489F4D8
:10552000103399F5D3018C918F7D883509F0B2C085
:1055300011961C91B2E06B0E711C026050E1E52ED9
:10554000F12CEAE0EE16F10409F4B0C0F0E1EF1638
:10555000F104D9F028E0E216F10451F438E0E32E2A
:10556000F12C88248A94982CA82C4FE1B42E13C0D7
:105570006FEF7FEFCB0197010F2C000C440B550B05
:105580000E94BC2E49015A0106C088248A94982C96
:10559000A82C2FE0B22E7E826D8260E020E030E009
:1055A000A90127010F2C000C660877082D803E808A
:1055B000E0EDE10FEA3060F08FEB810F8A3110F4FB
:1055C000E9EC05C08FE9810F8A3190F5E9EAE10F36
:1055D0008E2F90E08E159F055CF56F3F09F18216C6
:1055E0009306A406B506D8F0C301B2010E94AC2E02
:1055F0002E2F30E040E050E029833A834B835C83D8
:10560000260F371F481F591F89819A81AB81BC81A2
:10561000281739074A075B0710F061E001C06FEFF8
:10562000ED81FE813196FE83ED83D1011C91BECFC9
:10563000C114D10489F0662339F08D819E810197D0
:10564000F6019183808308C001FF06C08D819E8191
:105650000297D6018D939C9300FF07C0509540950B
:10566000309521953F4F4F4F5F4F67FF10C082E24B
:1056700090E090936206809361066FEF7FEF8FEF6B
:105680009FEF1BC060E070E080E090E016C0B901C1
:10569000CA0113C010E3E114F10409F45FCF51CF44
:1056A000103309F43FCF9AE0E92EF12C89E9882ED6
:1056B000982CA82C89E1B82E6ECF2696E2E10C94A6
:1056C000052FFC0188279927E89421912032E9F3DE
:1056D000293010F02E30C8F32B3241F02D3239F43E
:1056E000689404C00E94FB2B820F911D21912053CE
:1056F0002A30C0F31EF4909581959F4F08951F9313
:10570000FC0199278827BC01E89411911032E9F334
:10571000193010F01E30C8F31B3251F01D3249F41D
:10572000689406C00E94E62B610F711D811D911DBA
:10573000119110531A30B0F33EF490958095709506
:1057400061957F4F8F4F9F4F1F91089591110C943A
:10575000832E803219F089508550C8F708954BE5A3
:1057600056E00E94B42B0895FA01A191B0810097F0
:1057700019F41097E1F0CD01DC01CD010D9000206E
:1057800011F4C00113C0FB012191222319F020154F
:10579000D9F7F3CFFB012191201519F41E92119630
:1057A00006C02223C1F70D900020A1F7D001FA0115
:1057B000A193B0830895BB274A3031F4992322F492
:1057C000BDE2909581959F4F0C94042C592F482F42
:1057D000372F262F660F771F881F991F660F771F99
:1057E000881F991F620F731F841F951F660F771FF5
:1057F000881F991F08957AE0979F902D879F802D8D
:10580000910D11240895BB27FB015527AA27880F66
:10581000991FAA1FA41710F0A41B83955051B9F724
:10582000A05DAA3308F0A95DA193009779F7B111A3
:10583000B1931192CB010C94862E4F925F926F928E
:105840007F929F92AF92BF92CF92DF92EF92FF92A0
:105850000F931F93CF93DF93CDB7DEB729970FB682
:10586000F894DEBF0FBECDBF6A01122FB02E2BE31E
:10587000201720F0FF24F394F00E02C0BCE3FB2EAF
:105880000F2D27E0AE014F5F5F4F0E94AB2DAC01A3
:105890008981982F9970913031F0E1FC06C0E0FECB
:1058A00006C090E205C09DE203C09BE201C090E00B
:1058B000EE2DE07183FF3CC0911102C083E001C076
:1058C00084E0811718F4212F281B01C020E0E1118A
:1058D0000BC0F601822F30E2882319F031938150FA
:1058E000FBCFC20ED11C20E0992329F0D6019C9356
:1058F000F60131966F01C6010396E2FE0AC03EE44E
:10590000D6013C9341E411964C93119712963C9327
:1059100006C03EE6F601308341E641833283FC0156
:10592000322F40E2332309F442C041933150FACF81
:1059300082FF44C0911102C083E001C084E081175E
:1059400018F4212F281B01C020E0E1110BC0F60143
:10595000822F30E2882319F031938150FBCFC20EA1
:10596000D11C20E0992329F0D6019C93F6013196B1
:105970006F01C6010396E2FE0BC039E4D6013C93E9
:105980003EE411963C93119736E412963C9307C07F
:1059900039E6F60130833EE6318336E63283FC0198
:1059A000322F40E2332319F041933150FBCFFC01F9
:1059B000E20FF11D10828EEF9FEFB7C0F1E0911161
:1059C00001C0F0E06F2F70E01416150624F49A0160
:1059D0002F5F3F4F02C021E030E0260F371FBB2072
:1059E00029F06B2D70E06F5F7F4F02C060E070E0C8
:1059F000260F371F612F70E0261737071CF4121B84
:105A0000212F01C020E03E2D387159F4D601322FEC
:105A100060E2332319F06D933150FBCFC20ED11CDD
:105A200020E0FF2331F0D6019C93B6016F5F7F4FDA
:105A30006B01E1110BC0F601922F30E3992319F0AD
:105A400031939150FBCFC20ED11C20E09F2D940FBB
:105A50003A81782F7071A72E84FF03C0313309F487
:105A60009150191624F4993018F098E001C091E093
:105A7000E42F852F57FF02C0E0E080E06E2F782FE3
:105A8000E0E0F0E0AEE29A2E3A01691A71082A01CC
:105A9000461A570A0B2D10E01195019511096F3F19
:105AA0008FEF780729F4D6019C92C60101966C010C
:105AB0004617570784F0661677066CF47F01E40CEE
:105AC000F51CA1E0B0E0AC0FBD1FEA0EFB1ED70134
:105AD0001196BC9002C090E3B92E615071093196C5
:105AE000C60101967C016017710724F0D601BC92B3
:105AF0006C01D5CF6417750741F4363320F4353384
:105B000021F4A11002C081E3B82EF601B082F701A2
:105B1000822F90E2882319F091938150FBCFF701F7
:105B2000E20FF11D108280E090E029960FB6F89404
:105B3000DEBF0FBECDBFDF91CF911F910F91FF90C0
:105B4000EF90DF90CF90BF90AF909F907F906F903D
:105B50005F904F900895283008F027E03327DA014E
:105B6000990F311D87FD916000966105710539F42B
:105B700032602E5F3D9330E32A95E1F708959F3F11
:105B800030F080387105610509F03C5F3C5F3D9362
:105B9000913008F08068911DDF93CF931F930F938E
:105BA000FF92EF92192F987F9695E92F96959695EB
:105BB000E90FFF27EE52FF4F99273327EE24FF24EA
:105BC000A701E70105900894079428F4360FE71E13
:105BD000F81E491F511D660F771F881F991F0694D5
:105BE000A1F70590079428F4E70EF81E491F561FE9
:105BF000C11D770F881F991F661F0694A1F7059096
:105C0000079428F4F80E491F561FC71FD11D880F8F
:105C1000991F661F771F0694A1F70590079420F43B
:105C2000490F561FC71FD81F990F661F771F881F60
:105C30000694A9F784911095177041F0D695C795F1
:105C400057954795F794E7941A95C1F7E8E7F0E080
:105C500068941590159135916591959105907FE225
:105C60007395E118F10A430B560BC90BD009C0F725
:105C7000E10CF11E431F561FC91FD01D7EF4703367
:105C800011F48A95E6CFE894015030F0080F0AF439
:105C90000027021708F4202F2395022F7A3328F0CB
:105CA00079E37D932A95E9F710C07D932A9589F6CB
:105CB000069497956795379517951794E118F10A0B
:105CC000430B560BC90BD00998F023957E91739521
:105CD0007A3308F070E37C932013B8F77E917061FB
:105CE0007D9330F0839571E37D9370E32A95E1F71E
:105CF0001124EF90FF900F911F91CF91DF91992781
:105D000087FD90950895992788270895DC01FC0167
:105D1000672F71917723E1F7329704C07C916D93DF
:105D200070836291AE17BF07C8F30895F999FECF4B
:105D300092BD81BDF89A992780B50895262FF999CB
:105D4000FECF1FBA92BD81BD20BD0FB6F894FA9A5E
:105D5000F99A0FBE01960895DB018F939F930E94DD
:105D6000DE2EBF91AF91A29F800D911DA39F900D3C
:105D7000B29F900D11240895A1E21A2EAA1BBB1BFD
:105D8000FD010DC0AA1FBB1FEE1FFF1FA217B30707
:105D9000E407F50720F0A21BB30BE40BF50B661F1D
:105DA000771F881F991F1A9469F7609570958095E1
:105DB00090959B01AC01BD01CF0108950E94202F59
:105DC000A59F900DB49F900DA49F800D911D11244F
:105DD00008952F923F924F925F926F927F928F928F
:105DE0009F92AF92BF92CF92DF92EF92FF920F936A
:105DF0001F93CF93DF93CDB7DEB7CA1BDB0B0FB674
:105E0000F894DEBF0FBECDBF09942A883988488830
:105E10005F846E847D848C849B84AA84B984C884C6
:105E2000DF80EE80FD800C811B81AA81B981CE0FBD
:105E3000D11D0FB6F894DEBF0FBECDBFED010895A2
:105E4000A29FB001B39FC001A39F700D811D1124BB
:105E5000911DB29F700D811D1124911D0895505800
:105E6000BB27AA270E94472F0C94BA300E94AC305F
:105E700038F00E94B33020F039F49F3F19F426F433
:105E80000C94A9300EF4E095E7FB0C94A330E92FB5
:105E90000E94CB3058F3BA1762077307840795073F
:105EA00020F079F4A6F50C94ED300EF4E0950B2E6D
:105EB000BA2FA02D0B01B90190010C01CA01A0015C
:105EC0001124FF27591B99F0593F50F4503E68F1B7
:105ED0001A16F040A22F232F342F4427585FF3CFF8
:105EE000469537952795A795F0405395C9F77EF4C9
:105EF0001F16BA0B620B730B840BBAF09150A1F012
:105F0000FF0FBB1F661F771F881FC2F70EC0BA0F97
:105F1000621F731F841F48F4879577956795B7951F
:105F2000F7959E3F08F0B0CF9395880F08F099271A
:105F3000EE0F9795879508950E947F3008F481E0D1
:105F400008950E94B52F0C94BA300E94B33058F0D7
:105F50000E94AC3040F029F45F3F29F00C94A3304C
:105F600051110C94EE300C94A9300E94CB3068F3A0
:105F70009923B1F3552391F3951B550BBB27AA2702
:105F800062177307840738F09F5F5F4F220F331F3C
:105F9000441FAA1FA9F335D00E2E3AF0E0E832D004
:105FA00091505040E695001CCAF72BD0FE2F29D007
:105FB000660F771F881FBB1F261737074807AB07D9
:105FC000B0E809F0BB0B802DBF01FF2793585F4F4E
:105FD0003AF09E3F510578F00C94A3300C94EE30CB
:105FE0005F3FE4F3983ED4F3869577956795B79530
:105FF000F7959F5FC9F7880F911D9695879597F93B
:106000000895E1E0660F771F881FBB1F62177307B3
:106010008407BA0720F0621B730B840BBA0BEE1FC8
:1060200088F7E09508950E94D33088F09F5798F044
:10603000B92F9927B751B0F0E1F0660F771F881F8D
:10604000991F1AF0BA95C9F714C0B13091F00E94A7
:10605000ED30B1E008950C94ED30672F782F88274C
:10606000B85F39F0B93FCCF3869577956795B395CE
:10607000D9F73EF490958095709561957F4F8F4F3D
:106080009F4F0895E89409C097FB3EF49095809542
:10609000709561957F4F8F4F9F4F9923A9F0F92FEE
:1060A00096E9BB279395F695879577956795B7956C
:1060B000F111F8CFFAF4BB0F11F460FF1BC06F5F52
:1060C0007F4F8F4F9F4F16C0882311F096E911C064
:1060D000772321F09EE8872F762F05C0662371F085
:1060E00096E8862F70E060E02AF09A95660F771F99
:1060F000881FDAF7880F9695879597F90895990F75
:106100000008550FAA0BE0E8FEEF16161706E80781
:10611000F907C0F012161306E407F50798F0621BA2
:10612000730B840B950B39F40A2661F0232B242B77
:10613000252B21F408950A2609F4A140A6958FEF96
:10614000811D811D089597F99F6780E870E060E0E8
:1061500008959FEF80EC089500240A941616170600
:1061600018060906089500240A9412161306140648
:1061700005060895092E0394000C11F4882352F0AB
:10618000BB0F40F4BF2B11F460FF04C06F5F7F4F63
:106190008F4F9F4F089557FD9058440F551F59F04A
:1061A0005F3F71F04795880F97FB991F61F09F3F04
:1061B00079F087950895121613061406551FF2CF2D
:1061C0004695F1DF08C0161617061806991FF1CF7D
:1061D00086957105610508940895E894BB276627A4
:1061E0007727CB0197F908950E947F3008F48FEF4D
:1061F00008950E940C310C94BA300E94AC3038F0F3
:106200000E94B33020F0952311F00C94A3300C942D
:10621000A93011240C94EE300E94CB3070F3959F7E
:10622000C1F3950F50E0551F629FF001729FBB278D
:10623000F00DB11D639FAA27F00DB11DAA1F649F29
:106240006627B00DA11D661F829F2227B00DA11DDC
:10625000621F739FB00DA11D621F839FA00D611D62
:10626000221F749F3327A00D611D231F849F600D83
:10627000211D822F762F6A2F11249F5750409AF0AC
:10628000F1F088234AF0EE0FFF1FBB1F661F771F38
:10629000881F91505040A9F79E3F510580F00C9403
:1062A000A3300C94EE305F3FE4F3983ED4F3869530
:1062B00077956795B795F795E7959F5FC1F7FE2BA3
:1062C000880F911D9695879597F908950E947F30C4
:1062D000880B990B0895EE0FFF1F0590F491E02DA8
:1062E000099481E090E0F8940C94BB3191110895E9
:1062F00081568A5108F4805285580895FB01DC01CB
:1063000002C001900D9241505040D8F7089568178F
:10631000790768F4FB01DC01E40FF51FA40FB51F3A
:1063200002C002900E9241505040D8F708950C944C
:106330007E31DC0101C06D9341505040E0F708957B
:10634000FB01DC010D900020E9F7119701900D92FF
:106350000020E1F70895FB01DC018D910190801987
:106360000110D9F3990B0895FB01DC0101900D9206
:0A6370000020E1F70895F894FFCF34
:10637A000101FF00044D51545404FFFFFFFFFFFFCA
:10638A00DEEDBAFEFEED000000006112CE11F91139
:10639A00A8122A1208121C12000000007C034F03E4
:1063AA003A023902000000001A0715073A0267028A
:1063BA002003EB01970361072C02C60344071A0264
:1063CA002E0708022F0200000000851300000000BB
:1063DA001E13312E30003D003A00534156450054F9
:1063EA00454D5000484D445400494E413000494EF5
:1063FA00413100494E413200494E413300494E4134
:10640A003400494E4135004F555430004F555431F0
:10641A00004F555432004F555433004F55543400F1
:10642A004F555435002F006E616E00696E66006F1D
:10643A007666004448543031007465737475736528
:0E644A0072007465737470617373000D0A0044
:107E0000112484B714BE81FFF0D085E080938100F7
:107E100082E08093C00088E18093C10086E0809377
:107E2000C20080E18093C4008EE0C9D0259A86E02C
:107E300020E33CEF91E0309385002093840096BBD3
:107E4000B09BFECF1D9AA8958150A9F7CC24DD24C4
:107E500088248394B5E0AB2EA1E19A2EF3E0BF2EE7
:107E6000A2D0813461F49FD0082FAFD0023811F036
:107E7000013811F484E001C083E08DD089C08234E0
:107E800011F484E103C0853419F485E0A6D080C0E4
:107E9000853579F488D0E82EFF2485D0082F10E0AE
:107EA000102F00270E291F29000F111F8ED06801E7
:107EB0006FC0863521F484E090D080E0DECF843638
:107EC00009F040C070D06FD0082F6DD080E0C81688
:107ED00080E7D80618F4F601B7BEE895C0E0D1E017
:107EE00062D089930C17E1F7F0E0CF16F0E7DF06D8
:107EF00018F0F601B7BEE89568D007B600FCFDCFD4
:107F0000A601A0E0B1E02C9130E011968C91119780
:107F100090E0982F8827822B932B1296FA010C0160
:107F200087BEE89511244E5F5F4FF1E0A038BF0790
:107F300051F7F601A7BEE89507B600FCFDCF97BE46
:107F4000E89526C08437B1F42ED02DD0F82E2BD052
:107F50003CD0F601EF2C8F010F5F1F4F84911BD097
:107F6000EA94F801C1F70894C11CD11CFA94CF0C13
:107F7000D11C0EC0853739F428D08EE10CD085E9AC
:107F80000AD08FE07ACF813511F488E018D01DD067
:107F900080E101D065CF982F8091C00085FFFCCF94
:107FA0009093C60008958091C00087FFFCCF809118
:107FB000C00084FD01C0A8958091C6000895E0E648
:107FC000F0E098E1908380830895EDDF803219F02E
:107FD00088E0F5DFFFCF84E1DECF1F93182FE3DFCA
:107FE0001150E9F7F2DF1F91089580E0E8DFEE27F6
:047FF000FF270994CA
:027FFE00040479
:0400000300007E007B
:00000001FF
